BL51 BANKED LINKER/LOCATER V5.03                                                        08/02/2011  13:11:56  PAGE 1


BL51 BANKED LINKER/LOCATER V5.03, INVOKED BY:
C:\KEIL\C51\BIN\BL51.EXE DS1307.obj TO RTC RAMSIZE (256)


MEMORY MODEL: SMALL


INPUT MODULES INCLUDED:
  DS1307.obj (DS1307)
  C:\KEIL\C51\LIB\C51S.LIB (?C_STARTUP)
  C:\KEIL\C51\LIB\C51S.LIB (?C?CLDPTR)
  C:\KEIL\C51\LIB\C51S.LIB (?C?LMUL)
  C:\KEIL\C51\LIB\C51S.LIB (?C?SLCMP)


LINK MAP OF MODULE:  RTC (DS1307)


            TYPE    BASE      LENGTH    RELOCATION   SEGMENT NAME
            -----------------------------------------------------

            * * * * * * *   D A T A   M E M O R Y   * * * * * * *
            REG     0000H     0008H     ABSOLUTE     "REG BANK 0"
            DATA    0008H     0008H     UNIT         _DATA_GROUP_
            DATA    0010H     0007H     UNIT         ?DT?DS1307
            IDATA   0017H     0001H     UNIT         ?STACK

            * * * * * * *   C O D E   M E M O R Y   * * * * * * *
            CODE    0000H     0003H     ABSOLUTE     
            CODE    0003H     0085H     UNIT         ?PR?_DS1307_SET_TIME?DS1307
            CODE    0088H     0083H     UNIT         ?PR?DS1307_GET_TIME?DS1307
            CODE    010BH     007EH     UNIT         ?C?LIB_CODE
            CODE    0189H     007CH     UNIT         ?PR?MAIN?DS1307
            CODE    0205H     005AH     UNIT         ?PR?_DELAY_MS?DS1307
            CODE    025FH     003DH     UNIT         ?PR?LCD_INIT?DS1307
            CODE    029CH     0030H     UNIT         ?PR?_LCD_PRINT_B?DS1307
            CODE    02CCH     002FH     UNIT         ?PR?_I2C_WBYTE?DS1307
            CODE    02FBH     002FH     UNIT         ?PR?DS1307_INIT?DS1307
            CODE    032AH     0029H     UNIT         ?PR?I2C_ACK?DS1307
            CODE    0353H     0027H     UNIT         ?PR?I2C_RBYTE?DS1307
            CODE    037AH     0027H     UNIT         ?PR?_I2C_READ?DS1307
            CODE    03A1H     001CH     UNIT         ?PR?_LCD_PRINTXY?DS1307
            CODE    03BDH     001AH     UNIT         ?PR?_BIN2BCD?DS1307
            CODE    03D7H     0019H     UNIT         ?PR?_DELAY_US?DS1307
            CODE    03F0H     0019H     UNIT         ?PR?_I2C_WRITE?DS1307
            CODE    0409H     0019H     UNIT         ?PR?_BCD2BIN?DS1307
            CODE    0422H     0017H     UNIT         ?PR?_LCD_GOTOXY?DS1307
            CODE    0439H     0017H     UNIT         ?CO?DS1307
            CODE    0450H     0014H     UNIT         ?PR?I2C_START?DS1307
            CODE    0464H     0011H     UNIT         ?PR?LCD_DELAY?DS1307
            CODE    0475H     000EH     UNIT         ?PR?LCD_CLEAR?DS1307
            CODE    0483H     000EH     UNIT         ?PR?I2C_DELAY?DS1307
            CODE    0491H     000DH     UNIT         ?PR?I2C_STOP?DS1307
            CODE    049EH     000CH     UNIT         ?C_C51STARTUP
            CODE    04AAH     000BH     UNIT         ?PR?_LCD_COMMAND?DS1307
            CODE    04B5H     000BH     UNIT         ?PR?_LCD_PUTCHAR?DS1307
            CODE    04C0H     0008H     UNIT         ?PR?I2C_NACK?DS1307

BL51 BANKED LINKER/LOCATER V5.03                                                      08/02/2011  13:11:56  PAGE 2




OVERLAY MAP OF MODULE:   RTC (DS1307)


SEGMENT                               DATA_GROUP 
  +--> CALLED SEGMENT               START    LENGTH
---------------------------------------------------
?C_C51STARTUP                       -----    -----
  +--> ?PR?MAIN?DS1307

?PR?MAIN?DS1307                     -----    -----
  +--> ?PR?LCD_INIT?DS1307
  +--> ?PR?LCD_CLEAR?DS1307
  +--> ?PR?DS1307_INIT?DS1307
  +--> ?CO?DS1307
  +--> ?PR?_LCD_PRINTXY?DS1307
  +--> ?PR?_DELAY_MS?DS1307
  +--> ?PR?_DS1307_SET_TIME?DS1307
  +--> ?PR?DS1307_GET_TIME?DS1307
  +--> ?PR?_LCD_PRINT_B?DS1307
  +--> ?PR?_LCD_PUTCHAR?DS1307

?PR?LCD_INIT?DS1307                 -----    -----
  +--> ?PR?_LCD_COMMAND?DS1307
  +--> ?PR?_DELAY_MS?DS1307
  +--> ?PR?LCD_CLEAR?DS1307

?PR?_LCD_COMMAND?DS1307             -----    -----
  +--> ?PR?LCD_DELAY?DS1307

?PR?_DELAY_MS?DS1307                0008H    0008H

?PR?LCD_CLEAR?DS1307                -----    -----
  +--> ?PR?_LCD_COMMAND?DS1307
  +--> ?PR?LCD_DELAY?DS1307

?PR?DS1307_INIT?DS1307              -----    -----
  +--> ?PR?_I2C_READ?DS1307
  +--> ?PR?_BCD2BIN?DS1307
  +--> ?PR?_DELAY_US?DS1307
  +--> ?PR?_BIN2BCD?DS1307
  +--> ?PR?_I2C_WRITE?DS1307

?PR?_I2C_READ?DS1307                -----    -----
  +--> ?PR?I2C_START?DS1307
  +--> ?PR?I2C_ACK?DS1307
  +--> ?PR?_I2C_WBYTE?DS1307
  +--> ?PR?I2C_RBYTE?DS1307
  +--> ?PR?I2C_NACK?DS1307
  +--> ?PR?I2C_STOP?DS1307

?PR?I2C_START?DS1307                -----    -----
  +--> ?PR?I2C_DELAY?DS1307

?PR?I2C_ACK?DS1307                  -----    -----
  +--> ?PR?_I2C_WBYTE?DS1307
BL51 BANKED LINKER/LOCATER V5.03                                                      08/02/2011  13:11:56  PAGE 3


  +--> ?PR?I2C_DELAY?DS1307

?PR?_I2C_WBYTE?DS1307               -----    -----
  +--> ?PR?I2C_DELAY?DS1307

?PR?I2C_RBYTE?DS1307                -----    -----
  +--> ?PR?I2C_DELAY?DS1307

?PR?I2C_NACK?DS1307                 -----    -----
  +--> ?PR?I2C_DELAY?DS1307

?PR?I2C_STOP?DS1307                 -----    -----
  +--> ?PR?I2C_DELAY?DS1307

?PR?_I2C_WRITE?DS1307               -----    -----
  +--> ?PR?I2C_START?DS1307
  +--> ?PR?I2C_ACK?DS1307
  +--> ?PR?_I2C_WBYTE?DS1307
  +--> ?PR?I2C_STOP?DS1307

?PR?_LCD_PRINTXY?DS1307             -----    -----
  +--> ?PR?_LCD_GOTOXY?DS1307
  +--> ?PR?_LCD_PUTCHAR?DS1307

?PR?_LCD_GOTOXY?DS1307              -----    -----
  +--> ?PR?_LCD_COMMAND?DS1307

?PR?_LCD_PUTCHAR?DS1307             -----    -----
  +--> ?PR?LCD_DELAY?DS1307

?PR?_DS1307_SET_TIME?DS1307         0008H    0007H
  +--> ?PR?_BIN2BCD?DS1307
  +--> ?PR?_I2C_WRITE?DS1307

?PR?DS1307_GET_TIME?DS1307          -----    -----
  +--> ?PR?_I2C_READ?DS1307
  +--> ?PR?_BCD2BIN?DS1307

?PR?_LCD_PRINT_B?DS1307             -----    -----
  +--> ?PR?_LCD_PUTCHAR?DS1307



SYMBOL TABLE OF MODULE:  RTC (DS1307)

  VALUE           TYPE          NAME
  ----------------------------------

  -------         MODULE        DS1307
  C:0000H         SYMBOL        _ICE_DUMMY_
  C:04C0H         PUBLIC        i2c_nack
  D:0080H         PUBLIC        P0
  D:0090H         PUBLIC        P1
  D:00B0H         PUBLIC        P3
  C:0353H         PUBLIC        i2c_rbyte
  C:0335H         PUBLIC        i2c_ack
  C:0450H         PUBLIC        i2c_start
BL51 BANKED LINKER/LOCATER V5.03                                                      08/02/2011  13:11:56  PAGE 4


  C:03A7H         PUBLIC        _lcd_printxy
  C:0475H         PUBLIC        lcd_clear
  C:0422H         PUBLIC        _lcd_gotoxy
  C:0189H         PUBLIC        main
  C:0464H         PUBLIC        lcd_delay
  C:0491H         PUBLIC        i2c_stop
  D:0010H         PUBLIC        year
  C:020BH         PUBLIC        _delay_ms
  C:02FBH         PUBLIC        ds1307_init
  C:03D7H         PUBLIC        _delay_us
  D:0011H         PUBLIC        sec
  D:0012H         PUBLIC        day
  C:0003H         PUBLIC        _ds1307_set_time
  D:0013H         PUBLIC        min
  D:0014H         PUBLIC        mth
  D:0015H         PUBLIC        dow
  C:025FH         PUBLIC        lcd_init
  D:0016H         PUBLIC        hrs
  B:00B0H.4       PUBLIC        en
  C:0088H         PUBLIC        ds1307_get_time
  B:00B0H.6       PUBLIC        SDA
  C:04AAH         PUBLIC        _lcd_command
  C:037AH         PUBLIC        _i2c_read
  B:00B0H.7       PUBLIC        SCL
  B:00B0H.5       PUBLIC        rs
  C:029CH         PUBLIC        _lcd_print_b
  B:0080H.7       PUBLIC        SET
  C:03F0H         PUBLIC        _i2c_write
  C:02CCH         PUBLIC        _i2c_wbyte
  C:04B5H         PUBLIC        _lcd_putchar
  C:048AH         PUBLIC        i2c_delay
  C:0409H         PUBLIC        _bcd2bin
  C:03BDH         PUBLIC        _bin2bcd
  -------         PROC          _DELAY_US
  D:0006H         SYMBOL        us
  -------         DO            
  D:0004H         SYMBOL        z
  -------         ENDDO         
  C:03D7H         LINE#         9
  C:03D7H         LINE#         10
  C:03D7H         LINE#         12
  C:03DEH         LINE#         13
  C:03EFH         LINE#         14
  -------         ENDPROC       _DELAY_US
  -------         PROC          L?0070
  -------         ENDPROC       L?0070
  -------         PROC          _DELAY_MS
  D:0008H         SYMBOL        ms
  -------         DO            
  D:000CH         SYMBOL        j
  -------         ENDDO         
  C:020BH         LINE#         17
  C:0213H         LINE#         18
  C:0213H         LINE#         20
  C:0224H         LINE#         21
  C:025EH         LINE#         22
  -------         ENDPROC       _DELAY_MS
BL51 BANKED LINKER/LOCATER V5.03                                                      08/02/2011  13:11:56  PAGE 5


  -------         PROC          LCD_DELAY
  -------         DO            
  D:0007H         SYMBOL        a
  -------         ENDDO         
  C:0464H         LINE#         31
  C:0464H         LINE#         32
  C:0464H         LINE#         34
  C:0466H         LINE#         35
  C:046CH         LINE#         36
  C:046EH         LINE#         37
  C:0474H         LINE#         38
  -------         ENDPROC       LCD_DELAY
  -------         PROC          LCD_INIT
  C:025FH         LINE#         44
  C:025FH         LINE#         45
  C:025FH         LINE#         46
  C:0261H         LINE#         47
  C:0266H         LINE#         48
  C:026BH         LINE#         49
  C:0276H         LINE#         50
  C:027BH         LINE#         51
  C:0280H         LINE#         52
  C:0285H         LINE#         53
  C:028AH         LINE#         54
  C:028DH         LINE#         55
  C:0292H         LINE#         56
  C:0297H         LINE#         57
  -------         ENDPROC       LCD_INIT
  -------         PROC          LCD_CLEAR
  C:0475H         LINE#         64
  C:0475H         LINE#         65
  C:0475H         LINE#         66
  C:047AH         LINE#         67
  C:047DH         LINE#         68
  C:0480H         LINE#         69
  -------         ENDPROC       LCD_CLEAR
  -------         PROC          _LCD_COMMAND
  D:0007H         SYMBOL        cmd
  C:04AAH         LINE#         76
  C:04AAH         LINE#         77
  C:04AAH         LINE#         78
  C:04ACH         LINE#         79
  C:04AEH         LINE#         80
  C:04B0H         LINE#         81
  C:04B2H         LINE#         82
  -------         ENDPROC       _LCD_COMMAND
  -------         PROC          _LCD_GOTOXY
  D:0007H         SYMBOL        x
  D:0005H         SYMBOL        y
  C:0422H         LINE#         89
  C:0422H         LINE#         90
  C:0422H         LINE#         92
  C:0428H         LINE#         93
  C:0428H         LINE#         94
  C:042AH         LINE#         95
  C:042AH         LINE#         96
  C:042EH         LINE#         97
BL51 BANKED LINKER/LOCATER V5.03                                                      08/02/2011  13:11:56  PAGE 6


  C:0432H         LINE#         99
  C:0438H         LINE#         100
  -------         ENDPROC       _LCD_GOTOXY
  -------         PROC          _LCD_PUTCHAR
  D:0007H         SYMBOL        value
  C:04B5H         LINE#         107
  C:04B5H         LINE#         108
  C:04B5H         LINE#         109
  C:04B7H         LINE#         110
  C:04B9H         LINE#         111
  C:04BBH         LINE#         112
  C:04BDH         LINE#         113
  -------         ENDPROC       _LCD_PUTCHAR
  -------         PROC          L?0071
  -------         ENDPROC       L?0071
  -------         PROC          _LCD_PRINTXY
  D:0007H         SYMBOL        x
  D:0005H         SYMBOL        y
  D:0001H         SYMBOL        text
  C:03A7H         LINE#         118
  C:03A7H         LINE#         119
  C:03A7H         LINE#         120
  C:03AAH         LINE#         121
  C:03B0H         LINE#         122
  C:03B0H         LINE#         123
  C:03B3H         LINE#         124
  C:03BAH         LINE#         125
  C:03BCH         LINE#         126
  -------         ENDPROC       _LCD_PRINTXY
  -------         PROC          _LCD_PRINT_B
  D:0005H         SYMBOL        val_a
  -------         DO            
  D:0004H         SYMBOL        temp_a
  -------         ENDDO         
  C:029CH         LINE#         132
  C:029EH         LINE#         133
  C:029EH         LINE#         136
  C:02A4H         LINE#         137
  C:02A6H         LINE#         138
  C:02A6H         LINE#         139
  C:02ACH         LINE#         140
  C:02ACH         LINE#         141
  C:02B1H         LINE#         142
  C:02B7H         LINE#         143
  C:02BEH         LINE#         144
  C:02C5H         LINE#         145
  -------         ENDPROC       _LCD_PRINT_B
  C:0485H         SYMBOL        L?0069
  -------         PROC          L?0068
  -------         ENDPROC       L?0068
  C:0485H         SYMBOL        L?0069
  -------         PROC          I2C_DELAY
  -------         DO            
  D:0007H         SYMBOL        a
  -------         ENDDO         
  C:048AH         LINE#         30
  C:048AH         LINE#         31
BL51 BANKED LINKER/LOCATER V5.03                                                      08/02/2011  13:11:56  PAGE 7


  C:048AH         LINE#         33
  C:0490H         LINE#         34
  -------         ENDPROC       I2C_DELAY
  -------         PROC          I2C_START
  C:0450H         LINE#         40
  C:0450H         LINE#         41
  C:0450H         LINE#         44
  C:0452H         LINE#         45
  C:0455H         LINE#         46
  C:0457H         LINE#         47
  C:045AH         LINE#         48
  C:045CH         LINE#         49
  C:045FH         LINE#         50
  C:0461H         LINE#         51
  -------         ENDPROC       I2C_START
  -------         PROC          I2C_STOP
  C:0491H         LINE#         58
  C:0491H         LINE#         59
  C:0491H         LINE#         61
  C:0493H         LINE#         62
  C:0493H         LINE#         63
  C:0493H         LINE#         64
  C:0496H         LINE#         65
  C:0498H         LINE#         66
  C:049BH         LINE#         67
  C:049DH         LINE#         68
  -------         ENDPROC       I2C_STOP
  -------         PROC          _I2C_WBYTE
  D:0005H         SYMBOL        i2c_wb
  -------         DO            
  D:0004H         SYMBOL        a
  -------         ENDDO         
  C:02CCH         LINE#         74
  C:02CEH         LINE#         75
  C:02CEH         LINE#         78
  C:02D0H         LINE#         79
  C:02D0H         LINE#         80
  C:02D2H         LINE#         81
  C:02D5H         LINE#         82
  C:02EDH         LINE#         83
  C:02EDH         LINE#         84
  C:02EFH         LINE#         85
  C:02F1H         LINE#         87
  C:02F1H         LINE#         88
  C:02F3H         LINE#         89
  C:02F3H         LINE#         90
  C:02F3H         LINE#         91
  C:02F3H         LINE#         92
  C:02F6H         LINE#         93
  C:02FAH         LINE#         95
  -------         ENDPROC       _I2C_WBYTE
  -------         PROC          I2C_RBYTE
  -------         DO            
  D:0005H         SYMBOL        a
  D:0006H         SYMBOL        b
  -------         ENDDO         
  C:0353H         LINE#         101
BL51 BANKED LINKER/LOCATER V5.03                                                      08/02/2011  13:11:56  PAGE 8


  C:0353H         LINE#         102
  C:0353H         LINE#         105
  C:0355H         LINE#         107
  C:0356H         LINE#         108
  C:0356H         LINE#         109
  C:0358H         LINE#         110
  C:035BH         LINE#         111
  C:035EH         LINE#         112
  C:035EH         LINE#         113
  C:036BH         LINE#         114
  C:036BH         LINE#         115
  C:036EH         LINE#         116
  C:0370H         LINE#         117
  C:0373H         LINE#         118
  C:0377H         LINE#         119
  C:0379H         LINE#         120
  -------         ENDPROC       I2C_RBYTE
  -------         PROC          L?0067
  -------         ENDPROC       L?0067
  -------         PROC          I2C_ACK
  -------         DO            
  D:0006H         SYMBOL        a
  -------         ENDDO         
  C:0335H         LINE#         126
  C:0335H         LINE#         127
  C:0335H         LINE#         130
  C:0338H         LINE#         131
  C:033AH         LINE#         132
  C:033DH         LINE#         133
  C:033DH         LINE#         134
  C:033DH         LINE#         135
  C:033DH         LINE#         136
  C:0340H         LINE#         139
  C:0343H         LINE#         140
  C:0348H         LINE#         141
  C:034BH         LINE#         142
  C:034DH         LINE#         143
  C:0350H         LINE#         144
  C:0352H         LINE#         145
  -------         ENDPROC       I2C_ACK
  -------         PROC          I2C_NACK
  C:04C0H         LINE#         151
  C:04C0H         LINE#         152
  C:04C0H         LINE#         154
  C:04C0H         LINE#         155
  C:04C0H         LINE#         156
  C:04C0H         LINE#         157
  C:04C3H         LINE#         158
  C:04C5H         LINE#         159
  -------         ENDPROC       I2C_NACK
  -------         PROC          _I2C_WRITE
  D:0006H         SYMBOL        id
  D:0001H         SYMBOL        add
  D:0002H         SYMBOL        dat
  C:03F0H         LINE#         166
  C:03F6H         LINE#         167
  C:03F6H         LINE#         168
BL51 BANKED LINKER/LOCATER V5.03                                                      08/02/2011  13:11:56  PAGE 9


  C:03F9H         LINE#         169
  C:03FBH         LINE#         170
  C:03FBH         LINE#         171
  C:03FBH         LINE#         172
  C:03FEH         LINE#         173
  C:0403H         LINE#         174
  C:0406H         LINE#         175
  -------         ENDPROC       _I2C_WRITE
  -------         PROC          _I2C_READ
  D:0002H         SYMBOL        id
  D:0001H         SYMBOL        add
  -------         DO            
  D:0006H         SYMBOL        rd
  -------         ENDDO         
  C:037AH         LINE#         182
  C:037EH         LINE#         183
  C:037EH         LINE#         185
  C:0381H         LINE#         186
  C:0383H         LINE#         187
  C:0383H         LINE#         188
  C:0383H         LINE#         189
  C:0386H         LINE#         190
  C:0389H         LINE#         191
  C:0390H         LINE#         192
  C:0393H         LINE#         193
  C:0398H         LINE#         194
  C:039BH         LINE#         195
  C:039EH         LINE#         196
  C:03A0H         LINE#         197
  -------         ENDPROC       _I2C_READ
  -------         PROC          DS1307_INIT
  -------         DO            
  D:0003H         SYMBOL        temp
  D:0003H         SYMBOL        temp1
  -------         ENDDO         
  C:02FBH         LINE#         23
  C:02FBH         LINE#         24
  C:02FBH         LINE#         26
  C:0304H         LINE#         27
  C:0309H         LINE#         28
  C:030CH         LINE#         29
  C:0313H         LINE#         30
  C:031AH         LINE#         31
  C:0321H         LINE#         32
  -------         ENDPROC       DS1307_INIT
  -------         PROC          _DS1307_SET_TIME
  D:0008H         SYMBOL        day
  D:0009H         SYMBOL        mth
  D:000AH         SYMBOL        year
  D:000BH         SYMBOL        dow
  D:000CH         SYMBOL        hrs
  D:000DH         SYMBOL        min
  D:000EH         SYMBOL        sec
  C:0003H         LINE#         37
  C:0009H         LINE#         38
  C:0009H         LINE#         39
  C:000CH         LINE#         40
BL51 BANKED LINKER/LOCATER V5.03                                                      08/02/2011  13:11:56  PAGE 10


  C:000FH         LINE#         42
  C:0016H         LINE#         43
  C:001DH         LINE#         44
  C:0024H         LINE#         45
  C:002BH         LINE#         46
  C:0032H         LINE#         47
  C:0039H         LINE#         48
  C:0040H         LINE#         50
  C:0049H         LINE#         51
  C:0052H         LINE#         52
  C:005BH         LINE#         53
  C:0064H         LINE#         54
  C:006DH         LINE#         55
  C:0076H         LINE#         56
  C:007FH         LINE#         57
  -------         ENDPROC       _DS1307_SET_TIME
  -------         PROC          DS1307_GET_TIME
  C:0088H         LINE#         62
  C:0088H         LINE#         63
  C:0088H         LINE#         64
  C:0091H         LINE#         65
  C:009AH         LINE#         66
  C:00A3H         LINE#         67
  C:00ACH         LINE#         68
  C:00B5H         LINE#         69
  C:00BEH         LINE#         70
  C:00C7H         LINE#         72
  C:00CAH         LINE#         73
  C:00CDH         LINE#         74
  C:00D0H         LINE#         75
  C:00D3H         LINE#         76
  C:00D6H         LINE#         77
  C:00D9H         LINE#         79
  C:00E0H         LINE#         80
  C:00E7H         LINE#         81
  C:00EEH         LINE#         82
  C:00F5H         LINE#         83
  C:00FCH         LINE#         84
  C:0103H         LINE#         85
  C:010AH         LINE#         86
  -------         ENDPROC       DS1307_GET_TIME
  -------         PROC          _BIN2BCD
  D:0007H         SYMBOL        bin_value
  -------         DO            
  D:0007H         SYMBOL        temp
  D:0006H         SYMBOL        retval
  -------         ENDDO         
  C:03BDH         LINE#         92
  C:03BDH         LINE#         93
  C:03BDH         LINE#         97
  C:03BDH         LINE#         98
  C:03BFH         LINE#         100
  C:03BFH         LINE#         101
  C:03BFH         LINE#         102
  C:03C7H         LINE#         103
  C:03C7H         LINE#         104
  C:03CBH         LINE#         105
BL51 BANKED LINKER/LOCATER V5.03                                                      08/02/2011  13:11:56  PAGE 11


  C:03CFH         LINE#         106
  C:03D1H         LINE#         108
  C:03D1H         LINE#         109
  C:03D4H         LINE#         110
  C:03D4H         LINE#         111
  C:03D4H         LINE#         112
  C:03D4H         LINE#         114
  C:03D6H         LINE#         115
  -------         ENDPROC       _BIN2BCD
  -------         PROC          _BCD2BIN
  D:0007H         SYMBOL        bcd_value
  -------         DO            
  D:0006H         SYMBOL        temp
  -------         ENDDO         
  C:0409H         LINE#         117
  C:0409H         LINE#         118
  C:0409H         LINE#         120
  C:040BH         LINE#         121
  C:0410H         LINE#         122
  C:0413H         LINE#         123
  C:0421H         LINE#         124
  -------         ENDPROC       _BCD2BIN
  -------         PROC          MAIN
  C:0189H         LINE#         19
  C:0189H         LINE#         20
  C:0189H         LINE#         22
  C:018CH         LINE#         23
  C:018FH         LINE#         25
  C:0192H         LINE#         27
  C:0199H         LINE#         28
  C:019DH         LINE#         29
  C:019FH         LINE#         31
  C:01A2H         LINE#         32
  C:01A2H         LINE#         33
  C:01B7H         LINE#         34
  C:01B7H         LINE#         37
  C:01B7H         LINE#         38
  C:01B7H         LINE#         40
  C:01BAH         LINE#         42
  C:01C1H         LINE#         43
  C:01C6H         LINE#         44
  C:01CBH         LINE#         45
  C:01D0H         LINE#         46
  C:01D5H         LINE#         47
  C:01DAH         LINE#         48
  C:01E5H         LINE#         49
  C:01EAH         LINE#         50
  C:01EFH         LINE#         51
  C:01F4H         LINE#         52
  C:01F9H         LINE#         53
  C:01FEH         LINE#         54
  C:0203H         LINE#         56
  -------         ENDPROC       MAIN
  -------         ENDMOD        DS1307

  -------         MODULE        ?C?CLDPTR
  C:010BH         PUBLIC        ?C?CLDPTR
BL51 BANKED LINKER/LOCATER V5.03                                                      08/02/2011  13:11:56  PAGE 12


  -------         ENDMOD        ?C?CLDPTR

  -------         MODULE        ?C?LMUL
  C:0124H         PUBLIC        ?C?LMUL
  -------         ENDMOD        ?C?LMUL

  -------         MODULE        ?C?SLCMP
  C:0173H         PUBLIC        ?C?SLCMP
  -------         ENDMOD        ?C?SLCMP

Program Size: data=24.0 xdata=0 code=1224
LINK/LOCATE RUN COMPLETE.  0 WARNING(S),  0 ERROR(S)
